:10000000009D000000020000C53A00000000000052
:1000100000000000000000000000000000000000E0
:10002000801878FFE4B8200118F6D8F99000007F16
:10003000007E07E4F0A3DFFCDEFA758120022F06C4
:10004000121328502474742B1214DBE0701B747488
:100050002BF582E434031211A925E025E02477F57D
:1000600082E43403F5831227F02200022B59EFD3E8
:100070009403500D1212ADF583E5822D121100E4A8
:10008000F0220002303775F00212282DE0FCA3E0C8
:10009000FD75F09AEFA42445F582E5F03400F58370
:1000A000EE75F00202282D25E025E02477F582E4A4
:1000B0003403F583E0F8A3E0F9A3E0FAA3E0FB90B2
:1000C0000383E0FCA3E0FDA3E0FEA3E0C39BFBEE03
:1000D0009AFAED99F9EC98F822EF2466FFEE34FED7
:1000E000FE7C007D0A12274C7D3212275EEF249A97
:1000F000FFEE3401FEEB75F002A42427F582E5F053
:100100003400F583229004B1E0FF9004B0E0FE7566
:10011000F09AA424A8F582E5F03400F583E5822F57
:10012000F582E43583F583229004B2E0FEA3E0FF7C
:100130009004B0E0FD75F09AA4247BF582E5F034DC
:1001400000F58322EF2424FFEE34FAFE7C007D0AC2
:1001500012274C7D1E12275EEF24DCFFEE3405FED5
:10016000EB75F002A42421F582E5F03400F583223A
:10017000F583E493FC740193FD75F002EFA424076A
:10018000F582E5F03402F583ECF0A3EDF09004A2E3
:10019000E022E0FCA3E0FDEF75F09AA42457F5827D
:1001A000E5F034002275F002EBA4241BF582E5F0A3
:1001B0003400F583E0FCA3E0FD75F002EBA4241508
:1001C000F582E5F03400F58322F5837401F09003A5
:1001D00083E0FCA3E0FDA3E0FEA3E0FFEB22E0252B
:1001E000E02470F582E4341AF583E493FE740193FD
:1001F000FFE4FCFDC30227DFF583E493FC74019365
:10020000FD75F002EFA422C39DFFEE9CFEE075F0A9
:100210009AA42469F582E5F03400F583229004A1C4
:10022000E0FE75F09AA42433F582E5F03400F583FE
:10023000EF75F00202282DE4900014F0900372F0A4
:10024000900419E0900373F054F0FFF0229004B092
:10025000E0FF75F09AA42445F582E5F03400229081
:1002600004B0E0FD75F09AA4248DF582E5F0340029
:10027000F583229004B075F09AE0FFA42433F58250
:10028000E5F03400F5832275F002EBA4241BF5821F
:10029000E5F03400F58322902EC9F07404902E4FBF
:1002A000F0902EC322F0A3F0A3F0A3F0A3F0A3F0EC
:1002B000A322E04401F0E4900014F0900372227550
:1002C000F002EC12282DE0FEA3E0FFD322EF75F040
:1002D00009A42489F582E4340322EF75F009A424EB
:1002E000EBF582E43402229004B1E0FF9004B0E028
:1002F00075F09AA4249FF582E5F0340022E4F075AD
:10030000F09AEEA424B1F582E5F03400229004B016
:10031000E0FFA3E0FD227428902EC9F0902E4E221B
:100320009004A3E02413F582E43402F58322F583DC
:1003300075F002EC12282DE4229004B4E0FDEF9D4C
:100340007480F86E9822EDF0CBEFCBEBD3940322C0
:1003500075F09AEEA424CCF582E5F03400227419ED
:100360002EF582E43402F58322EE8FF01227B37566
:10037000F09AED22902EC9F07408902E4FF0902E36
:10038000C322E0FCA3E0FD75F09A22E04406F09061
:1003900000147401F0227420902EC9F0902E4E2289
:1003A000E0FF25E024A4F582E43404F58322EB2564
:1003B000E02430F582E4341CF58322E0249FF582AA
:1003C000E43400F583E0640122900013E0FF900420
:1003D000A2E0C39F222401F582E5F0340222240D1D
:1003E000F582E5F0340222F583E4F07F0122E0FC9F
:1003F000A3E0FDEC541F22E4F0A3F075F09A22E094
:10040000FEA3E0C39D22C3EF94F6EE6480947F22A6
:10041000F583E0FCA3E0FD75F00222E4900499F07E
:100420009002297402F022E490021DF09002E4F0A0
:1004300022242DF582E5F034002275F024A424A4B2
:10044000F582E43403F5832275F024A42406F582B2
:10045000E43403F583229004B0E0FFA3E0FD22A47E
:1004600024A8F582E5F03400F583E58222F0741AC1
:100470002EF582E43402F583E4F022900373E090D9
:100480000419F02275F00402282DE0FF9004A5E085
:10049000FEEFC8EEC80822F582E43402F583222577
:1004A000E025E024A5F582E4340222F582E434025A
:1004B000F5832225E025E0244EF582E4340222F57E
:1004C00082E43402F5832225E025E0242FF582E43E
:1004D000340222F582E43400F5832225E025E0246D
:1004E00006F582E4340022F582E43402F583222505
:1004F000E025E02499F582E4340222F582E4340315
:10050000F58322902EC5E4F0902ECDF0A3F022F5D5
:1005100082E43402F58322940AEE6480948022748B
:1005200002F0902EC3744022E02416F582E43402D7
:10053000F58322902EC6F0902EC57401F022ECF0C7
:10054000A3EDF09004B0E0229004A3E004F0229028
:1005500004A3E0FF75F002A422F090021EF09002C6
:10056000E5F022E0FEA3E0FFC3EE940422EEF0A348
:10057000EFF0900499E022E49004A3F09004A3E04B
:10058000FFC394094003021806EF902EC87014E0D0
:10059000545FF0A3746AF0902EC3744AF0A3740100
:1005A000F0800EE044F0F0902EC37480F0A3740746
:1005B000F09004A3E0901A6793902ECAF0E49004A0
:1005C000A2F0900013E0FF9004A2E0FEC39F40035E
:1005D0000217FD74E82E1214EFE0FF9004A5F0E47A
:1005E000F5E2EFC39408503B7415121513C083C095
:1005F0008212146A8002C333D8FCD082D083F09078
:100600002ECD7401F0C083C082E0FFC8EEC8088020
:1006100002C333D8FCD082D083F0902EC074C1F0D6
:100620000217769004A5E024F8F07416121513C092
:1006300083C08212146A8002C333D8FCD082D08374
:10064000F0902ECE7401F0C083C082E0FFC8EEC8E7
:10065000088002C333D8FCD082D083F0EEB4050604
:10066000902EC97420F0EE640660030216DE90043A
:10067000A3E0FFB4010F74321212F87404F0902E4C
:10068000C37470804FEFB402071212F674048054E2
:10069000EFB4030F74301213787408F0902EC37403
:1006A000208031EFB404071212F674828036EFB462
:1006B000050D1213767404F0902EC374F0803AEF97
:1006C000B40618902EC9742AF0902E4E7401F09042
:1006D0002EC374C0F0A37406F08023EFB4070A128F
:1006E000137674081215018010EFB40811902EC90A
:1006F0007431F0902E4E1214FFF0A37405F0EE64E6
:100700000760030217709004A3E0FFB4010F742088
:1007100012127774F0F0A37404F0021770EFB402B1
:1007200010902EC9742AF0740112127D74C0021741
:100730006BEFB4030974301213547420804DEFB47E
:10074000040F902EC97428F0748212135A744080DA
:100750003AEFB4050974201213547440802DEFB49D
:10076000060E902EC97431F0902E4F1214FF801B8C
:10077000EFB4070974321212777470800EEFB40868
:100780000F902EC9742812127A7440F0A37405F0E9
:10079000902EC074C2F0E49004A4F0900001742E76
:1007A000F0A3E4F09004A2E024E81214EFE0900437
:1007B000A5F0123248E5E220E20C9004A4E004F037
:1007C000E0C394C840D553E2FB1214E39004A5E0C3
:1007D000FD75F002A4FFAEF0900002E02FF0900053
:1007E00001E03EF0ED901AA093FF900001E475F057
:1007F000021227C985F082F583121362EF12125B91
:10080000C083C0829004A3E0D082D083121081EC18
:10081000F0A3EDF09004A2E004F00215A29004A36E
:10082000E004F002155C90021F7401F0229004B005
:10083000EFF0A3EDF09004B47403F0ED70037402D4
:10084000F09004B0E0FF121178F583C083C082906D
:1008500004B1E0FED082D0831210661213DFFFEEE7
:100860009CFE9004B2F0A3EFF012375AC312131992
:100870004003021909121108C083C0829004B1E03C
:10088000FCD082D083121081121349121118EC127D
:1008900010811212A61214F74027121110C083C043
:1008A000829004B1E0FCD082D083121081E4F0A3E6
:1008B000F0ED121178F583EC121211E475F001805D
:1008C0002B1213E650299004B0E0FF121115C083DB
:1008D000C0829004B1E0FED082D083121081E4F097
:1008E000A3F012117712107E74FFF5F01227B312E5
:1008F00012ED12104E1212ED1234741212ED12316A
:10090000A8EF7003021A159004B1E0FF9004B0E064
:10091000FE1212D01210FBE4F0EF6003021A15125F
:100920001330F583E4F0021A159004B1E07029A3A6
:10093000E0FEA3E0FF12375AD31213194009121236
:10094000C71210FB7401F0121A4E40239004B0E05D
:1009500075F09A1213348012121A4E40121212C7F6
:10096000F583E5822FF582E43583F5837401F01277
:100970001108C083C0829004B1E0FCD082D0831201
:10098000108112134912111812129F9464EE6480A0
:1009900094804022121110C083C0829004B1E0FC08
:1009A000D082D0831210811213D7ED12117B121353
:1009B0000E75F0018031C3EF949CEE6480947F50FB
:1009C000299004B0E0FF121115C083C0829004B1D9
:1009D000E0FED082D083121081E4F0A3F0121177F0
:1009E00012107E74FFF5F01227B3C39004B2E064D6
:1009F00080948050341212ED12343D1212ED1231F7
:100A000055EF602B9004B0121230F583C083C08282
:100A10009004B1E0FED082D08312108112117212C4
:100A2000107EECF0A3EDF080061212ED12104E12C3
:100A300012ED1236C69004B0E0FF121178F583C0B3
:100A400083C0829004B1E0FED082D083121066E0B1
:100A5000FEA3E09004B01211E7C083C0829004B1FD
:100A6000E0D082D083121081EEF0A3EFF022900448
:100A7000B2E0FEA3E0FF12375A9004B4E0FDD3EFDA
:100A80009D7480F86E98223F3F3F3F3F3F3F3F3F7E
:100A9000003200321770012C025800640258000422
:100AA000001E000A000A000F0064000A000C000C7F
:100AB0000000000000000000000000000001010133
:100AC0000D0E0F030405060708090A0B0C000102AE
:100AD0000032003200320032003200320032003286
:100AE0000032003200320032003200320032003276
:100AF000003700370037003700370037003700373E
:100B0000003700370037003700370037003700372D
:100B10000028002800280028002800280028002895
:100B20000028002800280028002800280028002885
:100B3000002D002D002D002D002D002D002D002D4D
:100B4000002D002D002D002D002D002D002D002D3D
:100B50000050005000500050005000500050005015
:100B60000050005000500050005000500050005005
:100B700000550055005500550055005500550055CD
:100B800000550055005500550055005500550055BD
:100B90000046004600460046004600460046004625
:100BA0000046004600460046004600460046004615
:100BB000002D002D002D002D002D002D002D002DCD
:100BC000002D002D002D002D002D002D002D002DBD
:100BD00000C800C800C800C800C800C800C800C8D5
:100BE00000C800C800C800C800C800C800C800C8C5
:100BF00000CD00CD00CD00CD00CD00CD00CD00CD8D
:100C000000CD00CD00CD00CD00CD00CD00CD00CD7C
:100C100000BE00BE00BE00BE00BE00BE00BE00BEE4
:100C200000BE00BE00BE00BE00BE00BE00BE00BED4
:100C3000002D002D002D002D002D002D002D002D4C
:100C4000002D002D002D002D002D002D002D002D3C
:100C500000FA00FA00FA00FA00FA00FA00FA00FAC4
:100C600000FA00FA00FA00FA00FA00FA00FA00FAB4
:100C7000E49004A3F09004A3E0FDC394095023750D
:100C8000F002121259E0FAA3E0FB75F002EF121223
:100C900035F583EAF0A3EBF0E4FF12180D121528E6
:100CA00080D3E49004A2F0900013E0FF9004A2E04F
:100CB000C39F4003021E12121380E4F0A3F0EF253D
:100CC000E024AAF582E43404F583E4F0A3F0EF70A5
:100CD00003021E09E49004A3F09004A3E0FDC39472
:100CE0000950189004A2E0FF1221A89004A2E0FF8E
:100CF000A3E0FD12236D12152880DEE49004A3F01A
:100D00009004A3E0FFC394094003021D8C749F2F3D
:100D100012139E60189004A2E075F09A121334F535
:100D200083E0640160079002E7E0B401199004A237
:100D30001211EDC083C0829004A3E0D082D0831250
:100D40001081E4F0A3F09004A3E0FF60599004A2A6
:100D5000E0FE1211EE121210E0FCA3E0C39403ECCB
:100D600064809480501A75F09AEE1211F1C083C01D
:100D7000829004A3E0D082D083121081E4F0A3F02B
:100D80009004A2E0FF1211EEC083C0829004A3E0A1
:100D9000D082D083121081E0FCA3E0FDEF12138219
:100DA000EC8DF01227B3121528021CE09004A2E08B
:100DB000FF75F09AA42459F582E5F03400F583E03C
:100DC000FCA3E01211E012126CECF0A3EDF0900421
:100DD000A2121380E0FCA3E01211E012126CE0FEFC
:100DE000A3E02DFFEE3CFE9004A2E0FD75F00212A0
:100DF000119DEEF0A3EFF09004BBE0602CEDB40188
:100E00001275F00212119DE0FFA3E09002E1CFF015
:100E1000A3EFF0EDB4021275F00212119DE0FFA3F2
:100E2000E0900226CFF0A3EFF09004A2E004F002DD
:100E30001C87E490021FF0229004A2747EF0E4A3C9
:100E4000F0900013E0FE9004A3E0FFC39E40030275
:100E50001FD112350EEF6003121407121300E07059
:100E60007C12152F1213B51213F0EF1210D91213B2
:100E7000DFEE9C40409004A3E09004A2F012130423
:100E80007401F090021DE004F09002E4F09004A3DD
:100E9000E0FF24191213417401F012371E9004A3CD
:100EA000E0FF12372D9004A3E0FF1236319004A327
:100EB000E0FF1210209004A3E0FF1234DEEF600880
:100EC0009004A3121508E4F09004A3E0FF12353E4D
:100ED000EF7003021FC8E490021E021FC312152FF9
:100EE0001213BE1213F0EF1210D91213DFEE9C5042
:100EF00003021F8D9004A3E09004A2F012328FEF42
:100F00007003021FC8E4FF9004A3E0FE1212321225
:100F1000120E121362EE12117B12120EECF0A3ED00
:100F2000F00FEFB409E1121300E4F0900014E0FFB9
:100F30007009900372E07003021FDFEF601F9003DF
:100F400072E06019121217BF2003D38001C340055D
:100F5000E4900373F0900373E0440580489000141C
:100F6000E0601F900372E07019121218BF2003D3C3
:100F70008001C34005E4900373F0900373E04401E3
:100F80008023900014E07077900372E06071121279
:100F900017BF2003D38001C34005E4900373F09092
:100FA0000373E04404F0900419F0C28A229004A371
:100FB000E0FF121304E4F012374B9004A3E0FF1299
:100FC000360F9004A3E0FF12373C9004A3E0FF1219
:100FD00036539004A3E024191213417401F09002D7
:100FE0001EE004F09002E5F09004A3E004F0021E7D
:100FF000219004A2E0FF900222E06F6002EFF02255
:10100000CBEFCB121267E0FEA3E0FF121199E0FCD8
:10101000A3E0FDC39FEC9E50030220D9E42DFFEC1A
:101020003404FE121267E0FCA3E0FDC3EF9DFFEE67
:101030009C12113FEEF0A3EFF0121267E0FEA3E066
:10104000FF121199E0FCA3E0C39FFFEC9E1210D4A5
:10105000EEF0A3EFF012138EE493FE740193FF12EF
:1010600010D5E0FCA3E0FDD39FEC9E405B12138EF5
:10107000E493FE740193FFC3ED9FFFEC9EC313FE48
:10108000EF13FF12138E7401932FFFE4933E12109F
:10109000D412154D64036003022115EBB4010F1245
:1010A00010D6E0FFA3E0900224CFF0A3EFF0EB64B2
:1010B0000260030221151210D5E0FFA3E090038720
:1010C000CFF0A3EFF00221151210D5E0FEA3E0FF50
:1010D0007C007D6312274C0D12275E1210D512156D
:1010E0004DB4030BEBB40107E4900224F0A3F0EB42
:1010F000640270419003878039121199E0FEA3E0E9
:10110000FF121267E0FCA3E0C39FEC9EC39404753A
:10111000F002EB50121210D9E4F0A3F01211407457
:1011200004F0A3E4F0800E1210D9E4F0A3F0121141
:1011300040E4F0A3F0EB640170441210D51212A643
:10114000949AEE940140081210B9EEF0A3EFF01259
:1011500010D51213CE900423F0EDA3F0121140121B
:1011600012A694DCEE94054008121124EEF0A3EFD1
:10117000F01211401213CE900427F0EDA3F0EB64AF
:101180000270441210D51212A6949AEE94014008EF
:101190001210B9EEF0A3EFF01210D51213CE900496
:1011A00025F0EDA3F01211401212A694DCEE940586
:1011B0004008121124EEF0A3EFF01211401213CEEA
:1011C000900429F0EDA3F0229004B0EFF0A3EDF02D
:1011D0009004B47407F0ED603F90009FE0640170EC
:1011E0000280089004B112139B702D121253C08319
:1011F000C0829004B1E0FED082D083121066121536
:101200001E121244C083C0829004B1E0D082D08309
:10121000121081E4F0A3F0229004B0121230F58392
:10122000C083C0829004B1E0FED082D083121081CE
:10123000121362EFA42433F582E5F0340012107E1D
:101240001213DFFFEE9CFE9004B2F0A3EFF0123712
:101250005A9004B4E0FDC312131E40030222F6129A
:1012600010E5E06401703675F09AEE1211F1121279
:1012700010E0FEA3E0C3941EEE648094804003025D
:10128000233C121253C083C0829004B1E0FED0828E
:10129000D083121066ECF0A3EDF002233C9004B270
:1012A000E0FEA3E0FF12123FC083C0829004B1E0D1
:1012B000FCD082D0831210811213491212471212ED
:1012C0009F1214F7402212123FC083C0829004B1D3
:1012D000E0FCD082D0831210811213D7ED121235A8
:1012E00012130E75F00180281213E6506F9004B0AF
:1012F000E0FF121244C083C0829004B1E0FED082AD
:10130000D083121081E4F0A3F012107174FFF5F095
:101310001227B302233C121253C083C0829004B13F
:10132000E0FED082D08312106612151EFF1211EE5D
:10133000C083C0829004B1E0FED082D083121081BD
:10134000E0FCA3E0C3941EEC64809480400E75F032
:101350009AEF12143F2E1211007401F01210E5E002
:10136000640170281212DF1210FBE0041212DE1268
:1013700010FBE0D3940540149004B1E0FF75F09A9F
:10138000EE1210F21212DD1210FBE4F0229004B003
:10139000EFF0A3EDF09004B47407F0ED7003740463
:1013A000F09002E7E064017002801290009FE06418
:1013B00001700280089004B112139B703A12122D32
:1013C000F583C083C0829004B1E0FED082D0831246
:1013D000108112117212107EECF0A3EDF09004B0A7
:1013E0001211EDC083C0829004B1E0D082D083128C
:1013F0001081E4F0A3F0229004B0E0FF121178F520
:1014000083C083C0829004B1E0FED082D0831210EA
:10141000661213DFFFEE9C9004B2F0A3EFF090048D
:10142000B0121508E06007E49004B2F0A3F0900455
:10143000B2E0FEA3E0FF12375A9004B4E0FDC312FD
:10144000131E40030224AE9004B2E0FEA3E0FF901E
:1014500004B0121113C083C0829004B1E0FCD082AA
:10146000D08312108112134912111812129F1214F4
:10147000F740259004B0121113C083C0829004B1CC
:10148000E0FCD082D0831210811213D7ED12117BB1
:1014900012130E75F001802B1213E650299004B040
:1014A000E0FF121115C083C0829004B1E0FED0822B
:1014B000D083121081E4F0A3F012117712107E7421
:1014C000FFF5F01227B312143612104E803AC39073
:1014D00004B2E064809480502F12143612343D120E
:1014E0001436123155EF602012122DF583C083C0DF
:1014F000829004B1E0FED082D0831210811211726A
:1015000012107EECF0A3EDF09004B0E0FF12117821
:10151000F583C083C0829004B1E0FED082D08312F4
:101520001066E0FEA3E09004B01211E7C083C08211
:101530009004B1E0D082D083121081EEF0A3EFF0DE
:1015400022E4FE900013E0FFEEC39F40030226CF8B
:1015500012133EE0640160030226CB74132E1213B3
:1015600006E0FC60030225F5EE6401704E121220C5
:10157000BF2003D38001C34005E4900373F09002C1
:10158000E5E0FD6401701B9002E4E0900373B40198
:1015900009E04409121295048015121292121539AD
:1015A0008016ED900373B4020BE0440512129512FD
:1015B000144D8004121292F012145BEE6402600368
:1015C0000226C4121220BF2003D38001C34005E4C9
:1015D000900373F09002E5E0FD6401701C9002E45A
:1015E000E0900373B4010612136BE48021E044041D
:1015F0001212951215390226C1ED900373B402053B
:10160000E044058003E04404F0E4900014F090030B
:1016100072F00226C1EC640160030226C4EE64018C
:101620007060121220BF2003D38001C34005E490F4
:101630000373F09002E4E0FFB4020B900373E04404
:101640000A12136E8013EF6401702690021EE09060
:101650000373B4010C12136BE490037212144D80E7
:101660001EE0440212136EE4900372F0121408801C
:101670000E900373E0440212136EE4900372F012B2
:10168000145BEE6402705D121220BF2003D3800150
:10169000C34005E4900373F09002E4E0B4021390B9
:1016A0000373E0440AF09003727401F0900014F0A8
:1016B000802F90021DE06401701C9002E5E0900311
:1016C00073B40105E044098013E044081212950444
:1016D000F0121407800B900373E044081212950473
:1016E000F012145B12133EE4F0C28A0E0225237F2F
:1016F0000422BB010689828A83E0225002E722BBD2
:10170000FE02E32289828A83E49322BB010CE582F4
:1017100029F582E5833AF583E0225006E92582F82F
:10172000E622BBFE06E92582F8E222E58229F5825F
:10173000E5833AF583E49322BB010689828A83F02C
:10174000225002F722BBFE01F322F8BB010DE58215
:1017500029F582E5833AF583E8F0225006E92582EF
:10176000C8F622BBFE05E92582C8F222EF8DF0A45F
:10177000A8F0CF8CF0A428CE8DF0A42EFE22BC00C1
:101780000BBE0029EF8DF084FFADF022E4CCF8759C
:10179000F008EF2FFFEE33FEEC33FCEE9DEC9840AB
:1017A00005FCEE9DFE0FD5F0E9E4CEFD22EDF8F547
:1017B000F0EE8420D21CFEADF075F008EF2FFFEDA7
:1017C00033FD4007985006D5F0F222C398FD0FD59F
:1017D000F0EA22C5F0F8A3E028F0C5F0F8E582159C
:1017E0008270021583E038F022A3F8E0C5F025F0FE
:1017F000F0E582158270021583E0C838F0E822EB2C
:101800009FF5F0EA9E42F0E99D42F0E89C45F02207
:10181000ECF0A3EDF0A3EEF0A3EFF022A882858315
:10182000F0D083D082122813122813122813122802
:1018300013E473E493A3C583C5F0C583C8C582C808
:10184000F0A3C583C5F0C583C8C582C822A425827C
:10185000F582E5F03583F58322EF4E6012EF6001EB
:101860000EEDBB010B89828A83F0A3DFFCDEFA2236
:1018700089F05007F709DFFCA9F022BBFEFCF30951
:10188000DFFCA9F02290049DE06006900499E0043A
:10189000F0900499E0B4010BE490049DF090049959
:1018A000E004F0900499E0B40320D3900225E09482
:1018B00064900224E09400500E900388E0946490B9
:1018C0000387E0940040031213FB90049CE0640142
:1018D00070589004A2F01213A940030229C0E0FF3F
:1018E00025E024D0F582E4341A121150FF25E024BB
:1018F000B0F582E4341A1211D81213B5121166FF32
:1019000025E024F0F582E4341A1211D81213BE1225
:101910001166FF25E02410F582E4341B1211D81261
:10192000141112116604F00228B6900417E0640145
:1019300070589004A2F01213A9504CE0FF25E02447
:10194000D0F582E4341B121150FF25E024B0F5825B
:10195000E4341B1211D81213B5121166FF25E024CE
:10196000F0F582E4341B1211D81213BE121166FF77
:1019700025E02410F582E4341C1211D8121411123F
:10198000116604F00229160229C0E49004A2F012A4
:1019900013A9504CE0FF25E02450F582E4341B12DB
:1019A0001150FF25E02430F582E4341B1211D812C7
:1019B00013B5121166FF25E02470F582E4341B1282
:1019C00011D81213BE121166FF25E02490F582E4AF
:1019D000341B1211D812141112116604F002296F6F
:1019E000900203A3E090041DF090041AE0B4AA034F
:1019F0001230F8900434E07011A3E0B4100CE490BD
:101A00000434F0A37410F01231FB227F051233CDA1
:101A1000EF600AE4900411F07F051237009002296C
:101A2000E024FE601814601E147003022AE32403ED
:101A30006003022B58121400E49002E3F090022994
:101A40007403F0022CC712155790021FE0700302B6
:101A50002ABC9002E3E004F0E49004A1F0900013AB
:101A6000E0FF9004A1E0C39F5072E4FF1211FD1249
:101A70001362EE12117B12120EECF0A3EDF01211B4
:101A8000FD121362EE12123512120EECF0A3EDF0FD
:101A90000FEFB409D79004A1E0FF1210D6E4F0A331
:101AA000F0EF1211417404F0A3E4F0EFB40110E47C
:101AB000900423F0A3F09004277404F0E4A3F0EF63
:101AC000B40210E4900425F0A3F09004297404F00B
:101AD000E4A3F09004A1E004F0022A3D9002E3E0C8
:101AE000C394035003022B58900012747EF0E490CC
:101AF0000220F09002E3F07F0E12370F900229745B
:101B000004F022900499E0B4020B7403F07F0412F5
:101B100037001235C3900499E0B403107F041233E8
:101B2000CDEF60087F041237001213FB1232481207
:101B3000155712324890021FE0603D121C50E4908D
:101B400004A1F0900013E0FE9004A1E0FFC39E50BA
:101B5000191233581233189004A1E0FF121FE0123B
:101B600032489004A1E004F080D912356E121E189C
:101B7000122521900229EFF022C0E0C083C082C06C
:101B8000D0E8C0E0E9C0E0EAC0E0EBC0E0EFC0E0D0
:101B9000D2AFE5DB30E415E5DB30E10280229004D2
:101BA00018E5DFF090049AE4F0022CACE5DB30E5B8
:101BB00005900414803EE5DB30E12CE5DB30E011DC
:101BC00090049E1234AE1234B71226EBF5DF022CCD
:101BD000AC90049BE064016003022CAC308A0302E9
:101BE0002CACD28A022CAC90049AE0700DA3E5DFF5
:101BF000F090049A7401F0022CAC90049BE0902FBA
:101C00004B93FFB4FF0F900418E5DFF090049BE0C6
:101C100004F0022CA6EF640F702F90049E1234AED5
:101C200090049BE0FF1234D5540F12271890049EA5
:101C30001234AE90049BE0FF04F01234D5FFE5DFD0
:101C400054F04F122718022CA690049E1234AE12A4
:101C500034B7E5DF12272A90049BE0FF6414704438
:101C6000E5DFB42025900411E06004E4F0800B90DF
:101C7000049D7401F0900499E4F090049C7401F0C8
:101C8000900417E4F090023B04F0E5DFB4101590E7
:101C9000049DE4F0900499F0900417F090049CF0F7
:101CA00090023BF0EFB4161EE5DFB4200B90041752
:101CB0007401F090049CE4F0E5DFB410099004177F
:101CC000E4F090049CF0900416E004F075DBFFD083
:101CD000E0FFD0E0FBD0E0FAD0E0F9D0E0F8D0D0DF
:101CE000D082D083D0E0327E027F0F7D007B017AEC
:101CF0000079151228391232D5122865E4FE9000B9
:101D000013E0FFEEC39F4003022D74E4FC75F09ACC
:101D1000EE1211181213101213D8EE1212D3F5830B
:101D2000E5822C121100E4F075F09AEE12124712BF
:101D300013101213D8EE12143F2C1211001212DDE0
:101D4000F583E5822C121100E4F0CFEECFCDECCD7F
:101D500012104E1236C60CEC640970B1121330F535
:101D600083E4F0CFEECF12371E12373C12372D121C
:101D7000374B74132E121306E4F012133EE4F09066
:101D8000021C747EF0E4A3F0A3F09002E4F0A3F050
:101D90000E022CDE900222747EF0900012F0E4908D
:101DA0000221F022E49004A3F0FF9004A2F0EF14CB
:101DB000601E14603514604C14605B2404707490D1
:101DC00004A47401F0A3742FF0A37458F0022E0D34
:101DD0001234AB9000011226EBFED3941F40031285
:101DE00034C41226D26E704B80431234AB90000282
:101DF0001226EBFED3940640031234C41226D26E90
:101E0000703180291234AB9000031226EBFE1226AB
:101E1000D26E701F80171234AB9000041226EBFEB6
:101E2000648B60031234C41226D26E70069004A232
:101E3000E004F00FEF64056003022D8E9004A2E031
:101E4000B40504A37401F09004A3E0FD60079004BE
:101E50002DE0547FF0CFEDCF22758A50538AEF905A
:101E600004B97411F09004B87422F09004BA743379
:101E7000F075997F759A80E4FFFEC29600000020FD
:101E8000970DD296000000309705E49004B9F00F4A
:101E9000BF00010EEF640A4E70E07590FF75993F28
:101EA000759AC0E4FEFF3096032097069004B8743C
:101EB00087F00FBF00010EEF640A4E70E9E4F5AD44
:101EC00075AEE075AF19F5AC7589FF75913E7599E2
:101ED0001FF59675931CF59BF595F592F59A75800F
:101EE0000CC289D28A9004BB04F022023394E4939A
:101EF000A3F8E493A34003F68001F208DFF48029FD
:101F0000E493A3F85407240CC8C333C4540F4420EB
:101F1000C8834004F456800146F6DFE4800B0102DA
:101F2000040810204080902FCBE47E019360BCA376
:101F3000FF543F30E509541FFEE493A360010ECF28
:101F400054C025E060A840B8E493A3FAE493A3F852
:101F5000E493A3C8C582C8CAC583CAF0A3C8C58212
:101F6000C8CAC583CADFE9DEE780BE0F000000FFF4
:101F7000FF00000000FFFFFFFFFFFFFFFFFF00006B
:101F80000000000000000000000000000000000051
:101F90000000000000000000000000000000000041
:101FA0000000000000000000000000000000000031
:101FB0000000000000000000000000000000000021
:101FC0000000000000000000000000000000000011
:101FD0000000000000000000000000000000000001
:101FE00000000000000000000000004102E300418A
:101FF0000228004102E60041001400410372004142
:102000000410004100000042022400004203870047
:102010000041023B0041022E004103730041022AAD
:10202000004102E70041049A0041049B004204126F
:10203000000041041400410416004104150041044D
:10204000181041049D00410499004104110141040C
:102050009C004104170000C0E0C0F0C083C082C0F3
:10206000D0E8C0E0ECC0E0EDC0E0EEC0E0EFC0E0E2
:10207000D2AF900228E004F0C3940A4021E4F0902B
:102080000383E0FCA3E0FDA3E0FEA3E02401FFE462
:102090003EFEE43DFDE43CFC9003831227F0D0E0DB
:1020A000FFD0E0FED0E0FDD0E0FCD0E0F8D0D0D012
:1020B00082D083D0F0D0E032902EC0E4F0902ECBCE
:1020C00074F4F0902F58E0540F24F0902EC8F09044
:1020D0002ECC7448F0902EC97428F0A3743FF09071
:1020E0002E407481121285F0A3F0A304121285749D
:1020F00002F0A3F0902EC67414F0902EC17490F0EC
:10210000A37401F0A37480F0A37407F043E31012EA
:102110003692900013EFF0229004A37408F0A3E429
:10212000F0A3743FF0A374DFF0E4FDFCF9758A10AE
:10213000538AEF0000009004A3E0FEA3E01234CB2A
:10214000FF69F90DBD00010CBC37EBBDDFE8900461
:10215000A5E0FEA3E0F5828E83E493697008900405
:102160001A7402F08005E490041AF0758A50538ABC
:10217000EF000000229004B6EDF09004B5EFF0A35C
:10218000E0FE1212ADF583E5822E121100E06035FB
:102190009004B5E012141AC083C0829004B6E0D057
:1021A00082D083121464121094901A821211CA40C1
:1021B000149004B6E0FF9004B5E01212AE1210FBCA
:1021C000E4F07F01227F00229004B6EDF09004B588
:1021D000EFF0A3E0FE1212BAF583E5822E12110091
:1021E000E060359004B5E0121428C083C0829004EA
:1021F000B6E0D082D083121464121094901A841224
:1022000011CA40149004B6E0FF9004B5E01212BB6E
:102210001210FBE4F07F01227F00227F007E08E4A1
:10222000FDFC9004A3F0A3F0758A10538AEF000020
:1022300000EF1234CBFB9004A4E02BF09004A3E059
:102240003400F00DBD00010CBC37E6BDE0E39004A6
:10225000A3E0FCA3E0FDEC900434F0EDA3F0758A5C
:1022600050538AEF0000002290022AE024FE601101
:102270001460252403703730883490022A7402F0E9
:102280002220882A90022A7403F09002E77401F059
:102290007F0E12370F0235E97F0E123405EF600E04
:1022A0007F0E12370FE490022AF09002E7F022909E
:1022B00004A4EFF0E0FF24741214DBE06034900219
:1022C0003BE06401700EEF121087901A761211CA6B
:1022D0004020800F9004A4E0121087901A7C121105
:1022E000CA400F9004A4E02474F582E4340312136E
:1022F000C7227F00227E007F807D007B017A0479E7
:10230000191228399004197405F0A37402F0E4A39B
:10231000F090042B74ABF090042D749DF09004B9F0
:10232000E090041FF09004B8E0900420F09004BA0C
:10233000E0900421F0022D849004BBE0603990020B
:10234000E1121543500EEF9400EE94034006900402
:10235000BA7487F0900226121543500EEF9400EEE7
:10236000940340069004BA7487F0E49004BBF090A4
:1023700004BAE0900421F022CBEFCBEB640170179C
:10238000121185E0900469F0121199A3E090046A9B
:10239000F0ECA3F0EDA3F0EB64027017121185E0EE
:1023A00090046DF0121199A3E090046EF0ECA3F08C
:1023B000EDA3F02275200153A87F122E3912359C0F
:1023C00043A8801236DA1236EE758DE0123675EFBC
:1023D00024E0600A2410700AC283C2828004D2837F
:1023E000D282122865438D201229EB80DF9004A24F
:1023F000EFF0C3940F502BE0FF248A121477E060B3
:1024000021EF12147F1210929004A21211BE400FFD
:102410009004A2E0248AF582E434021213C7227FDA
:1024200000227F00229004A6EFF0C3940F502BE00F
:10243000FF243C12148BE06021EF121493121092CF
:102440009004A61211BE400F9004A6E0243CF58231
:10245000E434021213C7227F00227F00229004B5C9
:10246000121326502E9004B5E0FFEB1212AE12109C
:10247000FBE0701FEB1212AE1210FB1211AB121424
:102480001AC083C0829004B5E0D082D08312146455
:102490001227F0229004B5121326502E9004B5E0B6
:1024A000FFEB1212BB1210FBE0701FEB1212BB12FB
:1024B00010FB1211AB121428C083C0829004B5E047
:1024C000D082D0831214641227F0229004A4E0FB7F
:1024D000A3E0FAA3E0F92290049BE0FF04F08F82CE
:1024E000758300229004A37401F0222DF582EE3C46
:1024F000F583E49322E92FF9E43AFA0226D2900414
:10250000A4EFF0E0FF242B12149FE0601EEF1214E2
:10251000A7121092901A721211CA400F9004A4E0F0
:10252000242BF582E434021213C7227F0022900488
:10253000A4EFF0E0FF24031214B3E0601EEF1214C6
:10254000BB121092901A7E1211CA400F9004A4E0A0
:102550002403F582E434001213C7227F0022900482
:10256000A4EFF0E0FF244B1214C7E0601EEF12143A
:10257000CF121092901A7E1211CA400F9004A4E05C
:10258000244BF582E434021213C7227F0022E4FFB9
:10259000FE900013E0FDEEC39D501BEF1210D6120B
:1025A00013F2EE1210D9E0FAA3E0D39DEA9C4003A7
:1025B000CFEECF0E80DB900223EFF02290049E74CA
:1025C00001F0A37404F0A37419F0E4F5DA75DA40AD
:1025D00043DA2075D74075DA5843A90875B80875ED
:1025E000F80822CBEFCBEBD3940F501C748A2B123C
:1025F0001477E07013748A2BF582E434021211A967
:1026000012147FF5831227F022CBEFCBEBD3940F7C
:10261000501C743C2B12148BE07013743C2BF5820D
:10262000E434021211A9121493F5831227F0221236
:102630001328501C742B2B12149FE07013742B2B37
:10264000F582E434021211A91214A7F5831227F0BF
:1026500022121328501C74032B1214B3E07013744D
:10266000032BF582E434001211A91214BBF5831276
:1026700027F022121328501C744B2B1214C7E07041
:1026800013744B2BF582E434021211A91214CFF506
:10269000831227F022E4FD900414E06011900419E5
:1026A000E0FE54F0FDEE540FF0E4900414F0CFED92
:1026B000CF221214E3FFFEEE901A9093600974E8A3
:1026C0002F1214EFEEF00F0EEEB410EB22900383F6
:1026D0001227FC000000007E007F0F7D007B017A46
:1026E00002793C022839EFD39403500D1212BAF547
:1026F00083E5822D121100E4F0227F0512370012CB
:1027000035C31230989002297401F0022CC775B2BB
:102710008E75B6F9E4F5B743B20143AA010236ADAE
:10272000EFD3940F5008748A2F121477E4F022EF3D
:10273000D3940F5008743C2F12148BE4F022EFD383
:1027400094035008742B2F12149FE4F022EFD394BB
:1027500003500874032F1214B3E4F022EFD3940350
:102760005008744B2F1214C7E4F022EFD394035097
:102770000874742F1214DBE4F022EE30E707C3E490
:102780009FFFE49EFE220000000000000000000009
:102790000000000000000000000000000000000039
:1027A0000000000000000000000000000000000029
:1027B0000000000000000000000000000000000019
:1027C0000000000000000000000000000000000009
:103010000000000000000000000000000000009020
:00000001FF
